:1000000000308A00662900000A108A100A1182074F
:1000100028340C34013406340A108A100A1182077D
:10002000413454342B3443344D3447344C343D3410
:1000300030340D3400340A108A100A1182070C344F
:100040004E3465346E34693420346E346F34763413
:100050006134203453344D34533420347A34703482
:100060007234613476346134213400340A108A10D9
:100070000A1182075A34613473346C346534743431
:100080006534203453344D34533420346E34613469
:1000900020346334693473346C346F3400340A10A0
:1000A0008A100A1182072034203420342034373457
:1000B0003334363420343634353435342034323425
:1000C0003534303400340A108A100A1182070C3497
:1000D0005034723469346A34613474346134203495
:1000E00053344D34533420347334203474346534F1
:1000F0007834743465346D3400340A108A100A116F
:100100008207413454342B3443344D34473444341F
:100110003D3431340D340034323084008313000810
:100120000319A3280130F800BF30F7006400F70B73
:100130009628F80B94284A30F700F70B9D2800000A
:100140006400800B922800340708F039B9003808A1
:100150000F39390487000614831606106400203016
:10016000F700F70BB128B428831206108316061087
:1001700083120034B608031DBF288610C0288614D9
:10018000831686108312B70E3708B800A420B70E66
:100190003708B800A42064004230F700F70BCE28DF
:1001A00000341430B2008C20F0308316870583129F
:1001B000861083168610831206108316061083128B
:1001C000AF012F08023C031CED280230B2008C2046
:1001D0000330B800A420AF0AE12864000C30F70017
:1001E000F70BF028F3280230B800A42064000C308C
:1001F000F700F70BF928FC28AF012F08023C031C7D
:100200000D292F080420B000B6013008B700BA202D
:100210000230B2008C20AF0AFD28B729013033022A
:10022000FC3E03182029043E2B29B401202940302C
:10023000B40020291430B40020295430B4002029FF
:1002400001303202B40734088038B500B6013508F1
:10025000B700BA2000340A148A100A11820715293F
:1002600017291A291D2931080C3A03194129063A80
:1002700003194929073A03194F29053A0319542943
:100280005929B6010130B700BA200230B2008C20E3
:1002900065290130B2000230B3000E21652901301A
:1002A000B200B3000E216529B6011030B700BA20A4
:1002B000652931081F3C031C5F290730B105013057
:1002C000B6003108B700BA206529003484018313D1
:1002D0001F3083050C3083169900A63098009030AB
:1002E0008312980083161F149F141F159F11073047
:1002F0009C00FF308312A00083161F149F141F154B
:100300009F1183121F108316091283129412A012D8
:100310002008831687008312201620088316870082
:100320008312A011200883168700013083129400E5
:100330000030831694000108C73908388100831201
:1003400090010030F80092000030831692000730D0
:100350009C00050864000230F700F70BAD29B029B6
:100360001C0883120D1383169D018312D128831656
:100370000512831205129630B2008C2083160512E6
:10038000831205169630B2008C2083160512831254
:1003900005129630B2008C208316051283120516C2
:1003A0009630B2008C20AF012F080C20AF0AF70066
:1003B00077080C1ED92999000A302F02031DD42971
:1003C0002130840083138403840A8C1EE5291A08D3
:1003D00080000D300002031DE42980018C1EEE29EF
:1003E0001A088C1EF1291A08213084008313840313
:1003F000840A8C1EF9291A0880000D300002031DA2
:10040000F829800121084F3C031D462A22084B3C55
:10041000031D462A0130B200B3000E21AF012F08A0
:100420001B20AF0AF700B100332116302F02031D45
:100430000F2A0130B2000230B3000E210130B200A9
:100440000330B3000E21AF012F083620AF0AF700AA
:10045000B100332114302F02031D242A0130B200D1
:100460000430B3000E21AF012F084F20AF0AF70070
:10047000B10033210F302F02031D342A1430AF0096
:10048000FA30B2008C20AF0B402A8A2BA901290830
:10049000363C031C502A8C1E4B2A1A08A90A472AEC
:1004A0002130840083138403840A8C1E552A1A0881
:1004B00080000D300002031D542A8001A108031D95
:1004C000632A3030A2003030A102A2022108093C88
:1004D00003186C2A0730A1022208093C0318722A6B
:1004E0000730A202A10EF030A1052208A104A30842
:1004F000031D7C2A3030A4003030A302A40223085C
:10050000093C0318852A0730A3022408093C031874
:100510008B2A0730A402A30EF030A3052408A304FD
:10052000A508031D952A3030A6003030A502A6028A
:100530002508093C03189E2A0730A5022608093C15
:100540000318A42A0730A602A50EF030A505260838
:10055000A504A708031DAE2A3030A8003030A7023A
:10056000A8022708093C0318B72A0730A702280861
:10057000093C0318BD2A0730A802A70EF030A705D2
:100580002808A7042308A2002508A3002708A40020
:10059000A701AB01A9012908033C031C3D2B031053
:1005A000AE0CAE17213029078400831300082E05F6
:1005B000AC0021302907F800FA010318FA0A78087C
:1005C000AF007A08B00021302907840083130008A7
:1005D000F7002B08F8000319F12A0310F70DF80BA8
:1005E000ED2A2F08840083133018831777088000C2
:1005F000AA012B08083C2A020318032B0310AD0C98
:10060000AD13AA0AF92A21302907F800FA010318C4
:10061000FA0A213029078400831300082D04B20050
:100620007808840083137A188317320880002130F9
:100630002907F800FA010318FA0A21302907840073
:10064000831300087F39B2007808840083137A1876
:100650008317320880002C08AD00AB0A2B08083C39
:10066000031D3B2BAB0101302907213E840083137E
:100670002D088000AE01A90ACB2A21302907840069
:10068000831380010130B2000230B3000E21AF01AC
:100690002F086320AF0AF700B100332115302F0275
:1006A000031D482B0930B2000330B3000E21213066
:1006B000840083130030000403196E2BB00104087A
:1006C000AF003010831B30140008B10033212F0815
:1006D0008400831330188317840A5A2B831605125B
:1006E000831205127830AF00FA30B2008C20AF0BC5
:1006F000742B8316051283120516AF012F087D2077
:10070000AF0AF70077080C1E832B99000A302F02DE
:08071000031D7E2BB7296300D5
:02400E00393F38
:00000001FF
